:020000040000FA
:100000000000000000000000000000008316C9305E
:1000100085008312073099008501A401A301E4281B
:10002000820733283E284B285A28692878288728B1
:100030009628A528B4280A30A1000000A00B1D288E
:10004000A10B1D2800340330A5000000A60B2528B5
:10005000A50B252800340530A5000000A60B2D288F
:10006000A50B2D2800348316E9308500831200305B
:1000700085002B20163085002B2000348316F930A4
:1000800085008312043085002B208316FF30850005
:1000900083122B2000348316CD308500831210305C
:1000A00085002B208316F9308500831202308500ED
:1000B0002B2000348316D930850083120030850050
:1000C0002B208316F93085008312063085002B2003
:1000D00000348316DB3085008312063085002B2028
:1000E0008316ED3085008312003085002B2000340C
:1000F0008316D93085008312023085002B208316A9
:10010000EB3085008312063085002B2000348316E7
:10011000C93085008312023085002B208316EB3016
:1001200085008312163085002B2000348316F930A9
:1001300085008312003085002B208316FD3085005A
:100140008312163085002B2000348316C9308500B9
:100150008312203085002B208316FD30850083120A
:10016000363085002B2000348316D9308500831269
:10017000003085002B208316E93085008312323051
:1001800085002B200034A4180129A414063023066E
:1001900003190129A30A0129A4180129A414013073
:1001A0002306031901290030230603190129A3039B
:1001B0000129A4180129A414063023060319E228F2
:1001C000A30A0129A30101298316FD3085008312AA
:1001D0000518ED28851DC328D928851DF328A401FD
:1001E00023081020E428A30AC3288316FD308500C5
:1001F00083120518FE28851DCC28D928851DC32803
:0C020000A40123081020F528FF23900023
:02400E00D43F9D
:00000001FF
